 saproc

 Timestamp is 62840d44 (reproducible build file hash)

 Preferred load address is 0000000180000000

 Start         Length     Name                   Class
 0001:00000000 00003700H .text$mn                CODE
 0001:00003700 00000036H .text$mn$00             CODE
 0001:00003736 0000010aH .text$x                 CODE
 0002:00000000 000001d8H .idata$5                DATA
 0002:000001d8 00000038H .00cfg                  DATA
 0002:00000210 00000008H .CRT$XCA                DATA
 0002:00000218 00000008H .CRT$XCZ                DATA
 0002:00000220 00000008H .CRT$XIA                DATA
 0002:00000228 00000008H .CRT$XIZ                DATA
 0002:00000230 00000008H .CRT$XPA                DATA
 0002:00000238 00000008H .CRT$XPZ                DATA
 0002:00000240 00000008H .CRT$XTA                DATA
 0002:00000248 00000008H .CRT$XTZ                DATA
 0002:00000250 00000000H .gehcont$y              DATA
 0002:00000250 00000000H .gfids$y                DATA
 0002:00000250 00000ab0H .rdata                  DATA
 0002:00000d00 00000000H .rdata$CastGuardVftablesA DATA
 0002:00000d00 00000000H .rdata$CastGuardVftablesC DATA
 0002:00000d00 00000324H .rdata$r                DATA
 0002:00001024 00000074H .rdata$voltmd           DATA
 0002:00001098 00000300H .rdata$zzzdbg           DATA
 0002:00001398 00000008H .rtc$IAA                DATA
 0002:000013a0 00000008H .rtc$IZZ                DATA
 0002:000013a8 00000008H .rtc$TAA                DATA
 0002:000013b0 00000008H .rtc$TZZ                DATA
 0002:000013b8 00000530H .xdata                  DATA
 0002:000018e8 000000f8H .xdata$x                DATA
 0002:000019e0 000003b0H .edata                  DATA
 0002:00001d90 000000b4H .idata$2                DATA
 0002:00001e44 00000014H .idata$3                DATA
 0002:00001e58 000001d8H .idata$4                DATA
 0002:00002030 000004a2H .idata$6                DATA
 0003:00000000 00000038H .data                   DATA
 0003:00000038 00000080H .data$r                 DATA
 0003:000000b8 00000098H .data$rs                DATA
 0003:00000150 00000658H .bss                    DATA
 0004:00000000 000003b4H .pdata                  DATA
 0005:00000000 00000060H .rsrc$01                DATA
 0005:00000060 00000328H .rsrc$02                DATA

  Address         Publics by Value              Rva+Base               Lib:Object

 0000:00000000       __AbsoluteZero             0000000000000000     <absolute>
 0000:00000000       ___safe_se_handler_count   0000000000000000     <absolute>
 0000:00000000       ___safe_se_handler_table   0000000000000000     <absolute>
 0000:00000000       __arm64x_extra_rfe_table   0000000000000000     <absolute>
 0000:00000000       __arm64x_extra_rfe_table_size 0000000000000000     <absolute>
 0000:00000000       __arm64x_native_entrypoint 0000000000000000     <absolute>
 0000:00000000       __arm64x_redirection_metadata 0000000000000000     <absolute>
 0000:00000000       __arm64x_redirection_metadata_count 0000000000000000     <absolute>
 0000:00000000       __dynamic_value_reloc_table 0000000000000000     <absolute>
 0000:00000000       __enclave_config           0000000000000000     <absolute>
 0000:00000000       __guard_check_icall_a64n_fptr 0000000000000000     <absolute>
 0000:00000000       __guard_eh_cont_count      0000000000000000     <absolute>
 0000:00000000       __guard_eh_cont_table      0000000000000000     <absolute>
 0000:00000000       __guard_fids_count         0000000000000000     <absolute>
 0000:00000000       __guard_fids_table         0000000000000000     <absolute>
 0000:00000000       __guard_iat_count          0000000000000000     <absolute>
 0000:00000000       __guard_iat_table          0000000000000000     <absolute>
 0000:00000000       __guard_longjmp_count      0000000000000000     <absolute>
 0000:00000000       __guard_longjmp_table      0000000000000000     <absolute>
 0000:00000000       __hybrid_auxiliary_delayload_iat 0000000000000000     <absolute>
 0000:00000000       __hybrid_auxiliary_delayload_iat_copy 0000000000000000     <absolute>
 0000:00000000       __hybrid_auxiliary_iat     0000000000000000     <absolute>
 0000:00000000       __hybrid_auxiliary_iat_copy 0000000000000000     <absolute>
 0000:00000000       __hybrid_code_map          0000000000000000     <absolute>
 0000:00000000       __hybrid_code_map_count    0000000000000000     <absolute>
 0000:00000000       __hybrid_image_info_bitfield 0000000000000000     <absolute>
 0000:00000000       __x64_code_ranges_to_entry_points 0000000000000000     <absolute>
 0000:00000000       __x64_code_ranges_to_entry_points_count 0000000000000000     <absolute>
 0000:00000100       __guard_flags              0000000000000100     <absolute>
 0000:00000000       __ImageBase                0000000180000000     <linker-defined>
 0001:00000000       Java_sun_jvm_hotspot_asm_Disassembler_decode 0000000180001000 f   sadis.obj
 0001:00000214       Java_sun_jvm_hotspot_asm_Disassembler_load_1library 0000000180001214 f   sadis.obj
 0001:000002c0       __local_stdio_printf_options 00000001800012c0 f i sadis.obj
 0001:00000520       ?AddRef@SAOutputCallbacks@@UEAAKXZ 0000000180001520 f   sawindbg.obj
 0001:00000530       ?CallObjectMethod@JNIEnv_@@QEAAPEAV_jobject@@PEAV2@PEAU_jmethodID@@ZZ 0000000180001530 f i sawindbg.obj
 0001:00000554       ?CallVoidMethod@JNIEnv_@@QEAAXPEAV_jobject@@PEAU_jmethodID@@ZZ 0000000180001554 f i sawindbg.obj
 0001:00000578       ?Output@SAOutputCallbacks@@UEAAJKPEBD@Z 0000000180001578 f   sawindbg.obj
 0001:00000628       ?QueryInterface@SAOutputCallbacks@@UEAAJAEBU_GUID@@PEAPEAX@Z 0000000180001628 f   sawindbg.obj
 0001:0000069c       ?Release@SAOutputCallbacks@@UEAAKXZ 000000018000169c f   sawindbg.obj
 0001:00001ac0       Java_sun_jvm_hotspot_debugger_windbg_WindbgDebuggerLocal_attach0__I 0000000180002ac0 f   sawindbg.obj
 0001:00001b20       Java_sun_jvm_hotspot_debugger_windbg_WindbgDebuggerLocal_attach0__Ljava_lang_String_2Ljava_lang_String_2 0000000180002b20 f   sawindbg.obj
 0001:00001b80       Java_sun_jvm_hotspot_debugger_windbg_WindbgDebuggerLocal_consoleExecuteCommand0 0000000180002b80 f   sawindbg.obj
 0001:00001e54       Java_sun_jvm_hotspot_debugger_windbg_WindbgDebuggerLocal_detach0 0000000180002e54 f   sawindbg.obj
 0001:00001eb4       Java_sun_jvm_hotspot_debugger_windbg_WindbgDebuggerLocal_getThreadIdFromSysId0 0000000180002eb4 f   sawindbg.obj
 0001:00001f38       Java_sun_jvm_hotspot_debugger_windbg_WindbgDebuggerLocal_initIDs 0000000180002f38 f   sawindbg.obj
 0001:000021f0       Java_sun_jvm_hotspot_debugger_windbg_WindbgDebuggerLocal_lookupByAddress0 00000001800031f0 f   sawindbg.obj
 0001:000022fc       Java_sun_jvm_hotspot_debugger_windbg_WindbgDebuggerLocal_lookupByName0 00000001800032fc f   sawindbg.obj
 0001:000023e8       Java_sun_jvm_hotspot_debugger_windbg_WindbgDebuggerLocal_readBytesFromProcess0 00000001800033e8 f   sawindbg.obj
 0001:000024ec       fprintf                    00000001800034ec f i sawindbg.obj
 0001:00002530       printf                     0000000180003530 f i sawindbg.obj
 0001:00002584       snprintf                   0000000180003584 f i sawindbg.obj
 0001:000025db       DebugCreate                00000001800035db f   dbgeng:dbgeng.dll
 0001:000025e1       JNU_ThrowByNameWithLastError 00000001800035e1 f   java:java.dll
 0001:000025e8       __GSHandlerCheck           00000001800035e8 f   MSVCRT:gshandler.obj
 0001:00002608       __GSHandlerCheckCommon     0000000180003608 f   MSVCRT:gshandler.obj
 0001:00002680       __chkstk                   0000000180003680 f   MSVCRT:chkstk.obj
 0001:00002680       _alloca_probe              0000000180003680 f   MSVCRT:chkstk.obj
 0001:000026e0       __security_check_cookie    00000001800036e0 f   MSVCRT:amdsecgs.obj
 0001:00002700       ??2@YAPEAX_K@Z             0000000180003700 f   MSVCRT:new_scalar.obj
 0001:0000273c       ??3@YAXPEAX_K@Z            000000018000373c f   MSVCRT:delete_scalar_size.obj
 0001:0000273c       ??_V@YAXPEAX@Z             000000018000373c f   MSVCRT:delete_array.obj
 0001:00002744       ??_U@YAPEAX_K@Z            0000000180003744 f   MSVCRT:new_array.obj
 0001:0000274c       __GSHandlerCheck_EH4       000000018000374c f   MSVCRT:gshandlereh4.obj
 0001:000027cc       ??_Etype_info@@UEAAPEAXI@Z 00000001800037cc f i MSVCRT:std_type_info_static.obj
 0001:000027cc       ??_Gtype_info@@UEAAPEAXI@Z 00000001800037cc f i MSVCRT:std_type_info_static.obj
 0001:00002b18       _DllMainCRTStartup         0000000180003b18 f   MSVCRT:dll_dllmain.obj
 0001:00002b58       __raise_securityfailure    0000000180003b58 f   MSVCRT:gs_report.obj
 0001:00002b8c       __report_gsfailure         0000000180003b8c f   MSVCRT:gs_report.obj
 0001:00002cd4       ??0bad_alloc@std@@QEAA@AEBV01@@Z 0000000180003cd4 f i MSVCRT:throw_bad_alloc.obj
 0001:00002d10       ??0bad_alloc@std@@QEAA@XZ  0000000180003d10 f i MSVCRT:throw_bad_alloc.obj
 0001:00002d30       ??0bad_array_new_length@std@@QEAA@AEBV01@@Z 0000000180003d30 f i MSVCRT:throw_bad_alloc.obj
 0001:00002d6c       ??0bad_array_new_length@std@@QEAA@XZ 0000000180003d6c f i MSVCRT:throw_bad_alloc.obj
 0001:00002d8c       ??0exception@std@@QEAA@AEBV01@@Z 0000000180003d8c f i MSVCRT:throw_bad_alloc.obj
 0001:00002dc0       ??1bad_alloc@std@@UEAA@XZ  0000000180003dc0 f i MSVCRT:throw_bad_alloc.obj
 0001:00002dc0       ??1bad_array_new_length@std@@UEAA@XZ 0000000180003dc0 f i MSVCRT:throw_bad_alloc.obj
 0001:00002dd4       ??_Ebad_alloc@std@@UEAAPEAXI@Z 0000000180003dd4 f i MSVCRT:throw_bad_alloc.obj
 0001:00002dd4       ??_Ebad_array_new_length@std@@UEAAPEAXI@Z 0000000180003dd4 f i MSVCRT:throw_bad_alloc.obj
 0001:00002dd4       ??_Eexception@std@@UEAAPEAXI@Z 0000000180003dd4 f i MSVCRT:throw_bad_alloc.obj
 0001:00002dd4       ??_Gbad_alloc@std@@UEAAPEAXI@Z 0000000180003dd4 f i MSVCRT:throw_bad_alloc.obj
 0001:00002dd4       ??_Gbad_array_new_length@std@@UEAAPEAXI@Z 0000000180003dd4 f i MSVCRT:throw_bad_alloc.obj
 0001:00002dd4       ??_Gexception@std@@UEAAPEAXI@Z 0000000180003dd4 f i MSVCRT:throw_bad_alloc.obj
 0001:00002e18       ?__scrt_throw_std_bad_alloc@@YAXXZ 0000000180003e18 f   MSVCRT:throw_bad_alloc.obj
 0001:00002e38       ?__scrt_throw_std_bad_array_new_length@@YAXXZ 0000000180003e38 f   MSVCRT:throw_bad_alloc.obj
 0001:00002e58       ?what@exception@std@@UEBAPEBDXZ 0000000180003e58 f i MSVCRT:throw_bad_alloc.obj
 0001:00002e6c       ??3@YAXPEAX@Z              0000000180003e6c f   MSVCRT:delete_scalar.obj
 0001:00002e74       __security_init_cookie     0000000180003e74 f   MSVCRT:gs_support.obj
 0001:00002f20       DllMain                    0000000180003f20 f   MSVCRT:dll_dllmain_stub.obj
 0001:00002f44       ?__scrt_initialize_type_info@@YAXXZ 0000000180003f44 f   MSVCRT:tncleanup.obj
 0001:00002f54       ?__scrt_uninitialize_type_info@@YAXXZ 0000000180003f54 f   MSVCRT:tncleanup.obj
 0001:00002f60       __local_stdio_scanf_options 0000000180003f60 f i MSVCRT:default_local_stdio_options.obj
 0001:00002f68       __scrt_initialize_default_local_stdio_options 0000000180003f68 f   MSVCRT:default_local_stdio_options.obj
 0001:00002f84       __scrt_acquire_startup_lock 0000000180003f84 f   MSVCRT:utility.obj
 0001:00002fc0       __scrt_dllmain_after_initialize_c 0000000180003fc0 f   MSVCRT:utility.obj
 0001:00002ff4       __scrt_dllmain_before_initialize_c 0000000180003ff4 f   MSVCRT:utility.obj
 0001:0000300c       __scrt_dllmain_crt_thread_attach 000000018000400c f   MSVCRT:utility.obj
 0001:00003034       __scrt_dllmain_crt_thread_detach 0000000180004034 f   MSVCRT:utility.obj
 0001:0000304c       __scrt_dllmain_exception_filter 000000018000404c f   MSVCRT:utility.obj
 0001:000030ac       __scrt_dllmain_uninitialize_c 00000001800040ac f   MSVCRT:utility.obj
 0001:000030dc       __scrt_dllmain_uninitialize_critical 00000001800040dc f   MSVCRT:utility.obj
 0001:000030f0       __scrt_initialize_crt      00000001800040f0 f   MSVCRT:utility.obj
 0001:0000313c       __scrt_initialize_onexit_tables 000000018000413c f   MSVCRT:utility.obj
 0001:000031c8       __scrt_is_nonwritable_in_current_image 00000001800041c8 f   MSVCRT:utility.obj
 0001:00003260       __scrt_release_startup_lock 0000000180004260 f   MSVCRT:utility.obj
 0001:00003284       __scrt_uninitialize_crt    0000000180004284 f   MSVCRT:utility.obj
 0001:000032b0       __scrt_get_dyn_tls_init_callback 00000001800042b0 f   MSVCRT:dyn_tls_init.obj
 0001:000032b8       __crt_debugger_hook        00000001800042b8 f   MSVCRT:utility_desktop.obj
 0001:000032c0       __scrt_fastfail            00000001800042c0 f   MSVCRT:utility_desktop.obj
 0001:0000340c       _RTC_Initialize            000000018000440c f   MSVCRT:initsect.obj
 0001:00003448       _RTC_Terminate             0000000180004448 f   MSVCRT:initsect.obj
 0001:00003484       _guard_check_icall_nop     0000000180004484 f i MSVCRT:guard_support.obj
 0001:00003488       __isa_available_init       0000000180004488 f   MSVCRT:cpu_disp.obj
 0001:00003634       _get_startup_argv_mode     0000000180004634 f   MSVCRT:argv_mode.obj
 0001:0000363c       __scrt_is_ucrt_dll_in_use  000000018000463c f   MSVCRT:ucrt_detection.obj
 0001:00003650       strchr                     0000000180004650 f   vcruntime:VCRUNTIME140.dll
 0001:00003656       __std_terminate            0000000180004656 f   vcruntime:VCRUNTIME140.dll
 0001:0000365c       memcmp                     000000018000465c f   vcruntime:VCRUNTIME140.dll
 0001:00003662       memset                     0000000180004662 f   vcruntime:VCRUNTIME140.dll
 0001:00003668       strstr                     0000000180004668 f   vcruntime:VCRUNTIME140.dll
 0001:0000366e       __CxxFrameHandler4         000000018000466e f   vcruntime:VCRUNTIME140_1.dll
 0001:00003674       __C_specific_handler       0000000180004674 f   vcruntime:VCRUNTIME140.dll
 0001:0000367a       __std_exception_copy       000000018000467a f   vcruntime:VCRUNTIME140.dll
 0001:00003680       __std_exception_destroy    0000000180004680 f   vcruntime:VCRUNTIME140.dll
 0001:00003686       _CxxThrowException         0000000180004686 f   vcruntime:VCRUNTIME140.dll
 0001:0000368c       __std_type_info_destroy_list 000000018000468c f   vcruntime:VCRUNTIME140.dll
 0001:00003692       strlen                     0000000180004692 f   ucrt:api-ms-win-crt-string-l1-1-0.dll
 0001:00003698       strcat                     0000000180004698 f   ucrt:api-ms-win-crt-string-l1-1-0.dll
 0001:0000369e       strcpy                     000000018000469e f   ucrt:api-ms-win-crt-string-l1-1-0.dll
 0001:000036a4       free                       00000001800046a4 f   ucrt:api-ms-win-crt-heap-l1-1-0.dll
 0001:000036aa       malloc                     00000001800046aa f   ucrt:api-ms-win-crt-heap-l1-1-0.dll
 0001:000036b0       _callnewh                  00000001800046b0 f   ucrt:api-ms-win-crt-heap-l1-1-0.dll
 0001:000036b6       _initterm                  00000001800046b6 f   ucrt:api-ms-win-crt-runtime-l1-1-0.dll
 0001:000036bc       _initterm_e                00000001800046bc f   ucrt:api-ms-win-crt-runtime-l1-1-0.dll
 0001:000036c2       _seh_filter_dll            00000001800046c2 f   ucrt:api-ms-win-crt-runtime-l1-1-0.dll
 0001:000036c8       _configure_narrow_argv     00000001800046c8 f   ucrt:api-ms-win-crt-runtime-l1-1-0.dll
 0001:000036ce       _initialize_narrow_environment 00000001800046ce f   ucrt:api-ms-win-crt-runtime-l1-1-0.dll
 0001:000036d4       _initialize_onexit_table   00000001800046d4 f   ucrt:api-ms-win-crt-runtime-l1-1-0.dll
 0001:000036da       _execute_onexit_table      00000001800046da f   ucrt:api-ms-win-crt-runtime-l1-1-0.dll
 0001:000036e0       _cexit                     00000001800046e0 f   ucrt:api-ms-win-crt-runtime-l1-1-0.dll
 0001:000036e8       __acrt_initialize          00000001800046e8 f   MSVCRT:ucrt_stubs.obj
 0001:000036e8       __acrt_thread_attach       00000001800046e8 f   MSVCRT:ucrt_stubs.obj
 0001:000036e8       __acrt_thread_detach       00000001800046e8 f   MSVCRT:ucrt_stubs.obj
 0001:000036e8       __acrt_uninitialize        00000001800046e8 f   MSVCRT:ucrt_stubs.obj
 0001:000036e8       __acrt_uninitialize_critical 00000001800046e8 f   MSVCRT:ucrt_stubs.obj
 0001:000036e8       __scrt_stub_for_acrt_initialize 00000001800046e8 f   MSVCRT:ucrt_stubs.obj
 0001:000036e8       __scrt_stub_for_acrt_thread_attach 00000001800046e8 f   MSVCRT:ucrt_stubs.obj
 0001:000036e8       __scrt_stub_for_acrt_thread_detach 00000001800046e8 f   MSVCRT:ucrt_stubs.obj
 0001:000036e8       __scrt_stub_for_acrt_uninitialize 00000001800046e8 f   MSVCRT:ucrt_stubs.obj
 0001:000036e8       __scrt_stub_for_acrt_uninitialize_critical 00000001800046e8 f   MSVCRT:ucrt_stubs.obj
 0001:000036e8       __vcrt_initialize          00000001800046e8 f   MSVCRT:ucrt_stubs.obj
 0001:000036e8       __vcrt_thread_attach       00000001800046e8 f   MSVCRT:ucrt_stubs.obj
 0001:000036e8       __vcrt_thread_detach       00000001800046e8 f   MSVCRT:ucrt_stubs.obj
 0001:000036e8       __vcrt_uninitialize        00000001800046e8 f   MSVCRT:ucrt_stubs.obj
 0001:000036e8       __vcrt_uninitialize_critical 00000001800046e8 f   MSVCRT:ucrt_stubs.obj
 0001:000036ec       __scrt_stub_for_is_c_termination_complete 00000001800046ec f   MSVCRT:ucrt_stubs.obj
 0001:000036ec       _is_c_termination_complete 00000001800046ec f   MSVCRT:ucrt_stubs.obj
 0001:000036ef       memcpy                     00000001800046ef f   vcruntime:VCRUNTIME140.dll
 0001:00003710       _guard_dispatch_icall_nop  0000000180004710 f   MSVCRT:guard_dispatch.obj
 0001:00003730       _guard_xfg_dispatch_icall_nop 0000000180004730 f   MSVCRT:guard_xfg_dispatch.obj
 0002:00000000       __imp_GetCurrentProcess    0000000180005000     kernel32:KERNEL32.dll
 0002:00000008       __imp_IsDebuggerPresent    0000000180005008     kernel32:KERNEL32.dll
 0002:00000010       __imp_GetProcAddress       0000000180005010     kernel32:KERNEL32.dll
 0002:00000018       __imp_LoadLibraryA         0000000180005018     kernel32:KERNEL32.dll
 0002:00000020       __imp_SwitchToThread       0000000180005020     kernel32:KERNEL32.dll
 0002:00000028       __imp_RtlCaptureContext    0000000180005028     kernel32:KERNEL32.dll
 0002:00000030       __imp_RtlLookupFunctionEntry 0000000180005030     kernel32:KERNEL32.dll
 0002:00000038       __imp_RtlVirtualUnwind     0000000180005038     kernel32:KERNEL32.dll
 0002:00000040       __imp_UnhandledExceptionFilter 0000000180005040     kernel32:KERNEL32.dll
 0002:00000048       __imp_SetUnhandledExceptionFilter 0000000180005048     kernel32:KERNEL32.dll
 0002:00000050       __imp_DisableThreadLibraryCalls 0000000180005050     kernel32:KERNEL32.dll
 0002:00000058       __imp_TerminateProcess     0000000180005058     kernel32:KERNEL32.dll
 0002:00000060       __imp_IsProcessorFeaturePresent 0000000180005060     kernel32:KERNEL32.dll
 0002:00000068       __imp_QueryPerformanceCounter 0000000180005068     kernel32:KERNEL32.dll
 0002:00000070       __imp_GetCurrentProcessId  0000000180005070     kernel32:KERNEL32.dll
 0002:00000078       __imp_GetCurrentThreadId   0000000180005078     kernel32:KERNEL32.dll
 0002:00000080       __imp_GetSystemTimeAsFileTime 0000000180005080     kernel32:KERNEL32.dll
 0002:00000088       __imp_InitializeSListHead  0000000180005088     kernel32:KERNEL32.dll
 0002:00000090       \177KERNEL32_NULL_THUNK_DATA 0000000180005090     kernel32:KERNEL32.dll
 0002:00000098       __imp___std_exception_destroy 0000000180005098     vcruntime:VCRUNTIME140.dll
 0002:000000a0       __imp___std_type_info_destroy_list 00000001800050a0     vcruntime:VCRUNTIME140.dll
 0002:000000a8       __imp_strchr               00000001800050a8     vcruntime:VCRUNTIME140.dll
 0002:000000b0       __imp___std_terminate      00000001800050b0     vcruntime:VCRUNTIME140.dll
 0002:000000b8       __imp_memcmp               00000001800050b8     vcruntime:VCRUNTIME140.dll
 0002:000000c0       __imp_memset               00000001800050c0     vcruntime:VCRUNTIME140.dll
 0002:000000c8       __imp_strstr               00000001800050c8     vcruntime:VCRUNTIME140.dll
 0002:000000d0       __imp__CxxThrowException   00000001800050d0     vcruntime:VCRUNTIME140.dll
 0002:000000d8       __imp___C_specific_handler 00000001800050d8     vcruntime:VCRUNTIME140.dll
 0002:000000e0       __imp___std_exception_copy 00000001800050e0     vcruntime:VCRUNTIME140.dll
 0002:000000e8       __imp_memcpy               00000001800050e8     vcruntime:VCRUNTIME140.dll
 0002:000000f0       \177VCRUNTIME140_NULL_THUNK_DATA 00000001800050f0     vcruntime:VCRUNTIME140.dll
 0002:000000f8       __imp___CxxFrameHandler4   00000001800050f8     vcruntime:VCRUNTIME140_1.dll
 0002:00000100       \177VCRUNTIME140_1_NULL_THUNK_DATA 0000000180005100     vcruntime:VCRUNTIME140_1.dll
 0002:00000108       __imp_free                 0000000180005108     ucrt:api-ms-win-crt-heap-l1-1-0.dll
 0002:00000110       __imp_malloc               0000000180005110     ucrt:api-ms-win-crt-heap-l1-1-0.dll
 0002:00000118       __imp_realloc              0000000180005118     ucrt:api-ms-win-crt-heap-l1-1-0.dll
 0002:00000120       __imp__callnewh            0000000180005120     ucrt:api-ms-win-crt-heap-l1-1-0.dll
 0002:00000128       \177api-ms-win-crt-heap-l1-1-0_NULL_THUNK_DATA 0000000180005128     ucrt:api-ms-win-crt-heap-l1-1-0.dll
 0002:00000130       __imp__initialize_onexit_table 0000000180005130     ucrt:api-ms-win-crt-runtime-l1-1-0.dll
 0002:00000138       __imp__initialize_narrow_environment 0000000180005138     ucrt:api-ms-win-crt-runtime-l1-1-0.dll
 0002:00000140       __imp__cexit               0000000180005140     ucrt:api-ms-win-crt-runtime-l1-1-0.dll
 0002:00000148       __imp__execute_onexit_table 0000000180005148     ucrt:api-ms-win-crt-runtime-l1-1-0.dll
 0002:00000150       __imp__initterm            0000000180005150     ucrt:api-ms-win-crt-runtime-l1-1-0.dll
 0002:00000158       __imp__initterm_e          0000000180005158     ucrt:api-ms-win-crt-runtime-l1-1-0.dll
 0002:00000160       __imp__seh_filter_dll      0000000180005160     ucrt:api-ms-win-crt-runtime-l1-1-0.dll
 0002:00000168       __imp__configure_narrow_argv 0000000180005168     ucrt:api-ms-win-crt-runtime-l1-1-0.dll
 0002:00000170       \177api-ms-win-crt-runtime-l1-1-0_NULL_THUNK_DATA 0000000180005170     ucrt:api-ms-win-crt-runtime-l1-1-0.dll
 0002:00000178       __imp___stdio_common_vfprintf 0000000180005178     ucrt:api-ms-win-crt-stdio-l1-1-0.dll
 0002:00000180       __imp___acrt_iob_func      0000000180005180     ucrt:api-ms-win-crt-stdio-l1-1-0.dll
 0002:00000188       __imp___stdio_common_vsprintf 0000000180005188     ucrt:api-ms-win-crt-stdio-l1-1-0.dll
 0002:00000190       \177api-ms-win-crt-stdio-l1-1-0_NULL_THUNK_DATA 0000000180005190     ucrt:api-ms-win-crt-stdio-l1-1-0.dll
 0002:00000198       __imp_strcpy               0000000180005198     ucrt:api-ms-win-crt-string-l1-1-0.dll
 0002:000001a0       __imp_strlen               00000001800051a0     ucrt:api-ms-win-crt-string-l1-1-0.dll
 0002:000001a8       __imp_strcat               00000001800051a8     ucrt:api-ms-win-crt-string-l1-1-0.dll
 0002:000001b0       \177api-ms-win-crt-string-l1-1-0_NULL_THUNK_DATA 00000001800051b0     ucrt:api-ms-win-crt-string-l1-1-0.dll
 0002:000001b8       __imp_DebugCreate          00000001800051b8     dbgeng:dbgeng.dll
 0002:000001c0       \177dbgeng_NULL_THUNK_DATA 00000001800051c0     dbgeng:dbgeng.dll
 0002:000001c8       __imp_JNU_ThrowByNameWithLastError 00000001800051c8     java:java.dll
 0002:000001d0       \177java_NULL_THUNK_DATA   00000001800051d0     java:java.dll
 0002:000001d8       __guard_check_icall_fptr   00000001800051d8     MSVCRT:guard_support.obj
 0002:000001e0       __guard_xfg_check_icall_fptr 00000001800051e0     MSVCRT:guard_support.obj
 0002:000001e8       __guard_dispatch_icall_fptr 00000001800051e8     MSVCRT:guard_support.obj
 0002:000001f0       __guard_xfg_dispatch_icall_fptr 00000001800051f0     MSVCRT:guard_support.obj
 0002:000001f8       __guard_xfg_table_dispatch_icall_fptr 00000001800051f8     MSVCRT:guard_support.obj
 0002:00000200       __castguard_check_failure_os_handled_fptr 0000000180005200     MSVCRT:guard_support.obj
 0002:00000208       __guard_memcpy_fptr        0000000180005208     vcruntime:softmemtag.obj
 0002:00000210       __xc_a                     0000000180005210     MSVCRT:initializers.obj
 0002:00000218       __xc_z                     0000000180005218     MSVCRT:initializers.obj
 0002:00000220       __xi_a                     0000000180005220     MSVCRT:initializers.obj
 0002:00000228       __xi_z                     0000000180005228     MSVCRT:initializers.obj
 0002:00000230       __xp_a                     0000000180005230     MSVCRT:initializers.obj
 0002:00000238       __xp_z                     0000000180005238     MSVCRT:initializers.obj
 0002:00000240       __xt_a                     0000000180005240     MSVCRT:initializers.obj
 0002:00000248       __xt_z                     0000000180005248     MSVCRT:initializers.obj
 0002:00000250       ??_C@_0BM@DBCALOPO@decode_instructions_virtual@ 0000000180005250     sadis.obj
 0002:00000270       ??_C@_0BG@MNACLANO@GetProcAddress?5failed@ 0000000180005270     sadis.obj
 0002:00000288       ??_C@_0CL@BJCJOPKP@sun?1jvm?1hotspot?1debugger?1Debugg@ 0000000180005288     sadis.obj
 0002:000002b8       ??_C@_0DP@IEGOKKOO@?$CILsun?1jvm?1hotspot?1asm?1Instructi@ 00000001800052b8     sadis.obj
 0002:000002f8       ??_C@_0M@IHKAILBK@handleEvent@ 00000001800052f8     sadis.obj
 0002:00000308       ??_C@_0DO@KENEIINN@?$CILsun?1jvm?1hotspot?1asm?1Instructi@ 0000000180005308     sadis.obj
 0002:00000348       ??_C@_08DCIFBHIL@rawPrint@ 0000000180005348     sadis.obj
 0002:00000358       ??_C@_0BD@JFADHEFE@Ljava?1lang?1String?$DL@ 0000000180005358     sawindbg.obj
 0002:00000370       ??_C@_09NDJHOMOJ@imagePath@ 0000000180005370     sawindbg.obj
 0002:00000380       ??_C@_0L@IBJLJICF@symbolPath@ 0000000180005380     sawindbg.obj
 0002:0000038c       ??_C@_01LELAEKIP@J@        000000018000538c     sawindbg.obj
 0002:00000390       ??_C@_0BA@ENOAPBEH@ptrIDebugClient@ 0000000180005390     sawindbg.obj
 0002:000003a0       ??_C@_0BB@FKGMCAMI@ptrIDebugControl@ 00000001800053a0     sawindbg.obj
 0002:000003b8       ??_C@_0BE@HEDMCBCH@ptrIDebugDataSpaces@ 00000001800053b8     sawindbg.obj
 0002:000003d0       ??_C@_0BJ@NECGJCMP@ptrIDebugOutputCallbacks@ 00000001800053d0     sawindbg.obj
 0002:000003f0       ??_C@_0BC@NFADOE@ptrIDebugAdvanced@ 00000001800053f0     sawindbg.obj
 0002:00000408       ??_C@_0BB@CGICJHBO@ptrIDebugSymbols@ 0000000180005408     sawindbg.obj
 0002:00000420       ??_C@_0BH@MKNGBFEC@ptrIDebugSystemObjects@ 0000000180005420     sawindbg.obj
 0002:00000438       ??_C@_0BI@HMPCDPNN@?$CILjava?1lang?1String?$DLJJ?$CJV@ 0000000180005438     sawindbg.obj
 0002:00000450       ??_C@_0O@BAEIOKDM@addLoadObject@ 0000000180005450     sawindbg.obj
 0002:00000460       ??_C@_04OHLIFDMD@?$CIJ?$CJV@ 0000000180005460     sawindbg.obj
 0002:00000468       ??_C@_09IDCNHNJH@addThread@ 0000000180005468     sawindbg.obj
 0002:00000480       ??_C@_0ED@MJCAPJHB@?$CILjava?1lang?1String?$DLJ?$CJLsun?1jvm?1h@ 0000000180005480     sawindbg.obj
 0002:000004c8       ??_C@_0BE@PHFCBNMF@createClosestSymbol@ 00000001800054c8     sawindbg.obj
 0002:000004dc       ??_C@_06FABFLPEO@?$CIJ?$FLJ?$CJV@ 00000001800054dc     sawindbg.obj
 0002:000004e8       ??_C@_0BM@LHHFOJLN@setThreadIntegerRegisterSet@ 00000001800054e8     sawindbg.obj
 0002:00000510       ??_7SAOutputCallbacks@@6B@ 0000000180005510     sawindbg.obj
 0002:00000530       _GUID_00000000_0000_0000_c000_000000000046 0000000180005530     sawindbg.obj
 0002:00000540       _GUID_4bf58045_d654_4c40_b0af_683090f356dc 0000000180005540     sawindbg.obj
 0002:00000550       ??_C@_0CA@CHBBHPBL@out?5of?5memory?5debugger?5output?$CB?6@ 0000000180005550     sawindbg.obj
 0002:00000570       _GUID_27fe5639_8407_4f47_8364_ee118fb08ac8 0000000180005570     sawindbg.obj
 0002:00000580       _GUID_5182e668_105e_416e_ad92_24ef800424ba 0000000180005580     sawindbg.obj
 0002:00000590       _GUID_88f7dfab_3ea7_4c3a_aefb_c4e8106173aa 0000000180005590     sawindbg.obj
 0002:000005a0       _GUID_f2df5f53_071f_47bd_9de6_5734c3fed689 00000001800055a0     sawindbg.obj
 0002:000005b0       _GUID_8c31e98c_983a_48a5_9016_6fe5d667a950 00000001800055b0     sawindbg.obj
 0002:000005c0       _GUID_6b86fe2c_2c4f_4f0c_9da2_174311acc327 00000001800055c0     sawindbg.obj
 0002:000005d0       ??_C@_0DG@KFKFAAAK@Windbg?5Error?3?5not?5able?5to?5creat@ 00000001800055d0     sawindbg.obj
 0002:00000608       ??_C@_0BA@IHFGPCFN@?$CFs?5?$CIhr?3?50x?$CF08X?$CJ@ 0000000180005608     sawindbg.obj
 0002:00000618       ??_C@_0CM@HMPHNLCI@Windbg?5Error?3?5not?5able?5to?5get?5I@ 0000000180005618     sawindbg.obj
 0002:00000648       ??_C@_0DH@MEIJIPLO@Windbg?5Error?3?5not?5able?5to?5get?5I@ 0000000180005648     sawindbg.obj
 0002:00000680       ??_C@_0DF@EJNGMFHL@Windbg?5Error?3?5not?5able?5to?5get?5I@ 0000000180005680     sawindbg.obj
 0002:000006b8       ??_C@_0DE@BLHEEHEB@Windbg?5Error?3?5not?5able?5to?5get?5I@ 00000001800056b8     sawindbg.obj
 0002:000006f0       ??_C@_0DK@CBFLKIDH@Windbg?5Error?3?5not?5able?5to?5get?5I@ 00000001800056f0     sawindbg.obj
 0002:00000730       ??_C@_0DC@OGBAOIMM@Windbg?5Error?3?5not?5able?5to?5get?5i@ 0000000180005730     sawindbg.obj
 0002:00000768       ??_C@_0DD@GMBHLNMH@Windbg?5Error?3?5not?5able?5to?5get?5s@ 0000000180005768     sawindbg.obj
 0002:000007a0       ??_C@_0CD@LLBBNFEA@Windbg?5Error?3?5OpenDumpFile?5fail@ 00000001800057a0     sawindbg.obj
 0002:000007c8       ??_C@_0CD@OHANEGIO@Windbg?5Error?3?5WaitForEvent?5fail@ 00000001800057c8     sawindbg.obj
 0002:000007f0       ??_C@_0CE@NLOIALLD@Windbg?5Error?3?5AttachProcess?5fai@ 00000001800057f0     sawindbg.obj
 0002:00000818       ??_C@_0CH@OOOMOIHO@Windbg?5Error?3?5GetNumberModules?5@ 0000000180005818     sawindbg.obj
 0002:00000840       ??_C@_0CP@GGPCODCJ@out?5of?5memory?5to?5allocate?5debug@ 0000000180005840     sawindbg.obj
 0002:00000870       ??_C@_0CK@OGHLJMOC@Windbg?5Error?3?5GetModuleParamete@ 0000000180005870     sawindbg.obj
 0002:000008a0       ??_C@_0CF@IPJIKFLG@Windbg?5Error?3?5GetModuleNames?5fa@ 00000001800058a0     sawindbg.obj
 0002:000008c8       ??_C@_0CH@DLOHNIAK@Windbg?5Error?3?5GetNumberThreads?5@ 00000001800058c8     sawindbg.obj
 0002:000008f0       ??_C@_0CG@KABLKJNP@out?5of?5memory?5to?5allocate?5threa@ 00000001800058f0     sawindbg.obj
 0002:00000918       ??_C@_0CK@FNPIPCCJ@Windbg?5Error?3?5GetThreadIdsByInd@ 0000000180005918     sawindbg.obj
 0002:00000948       ??_C@_0CH@DDGKENOM@Windbg?5Error?3?5SetCurrentThread?5@ 0000000180005948     sawindbg.obj
 0002:00000970       ??_C@_0CP@GPDFIPCF@Windbg?5Error?3?5GetCurrentThreadS@ 0000000180005970     sawindbg.obj
 0002:000009a0       ??_C@_0EC@GGBPHBOJ@WARNING?3?5GetThreadIdBySystemId?5@ 00000001800059a0     sawindbg.obj
 0002:000009e8       ??_C@_0CD@EHILJEIM@Windbg?5Error?3?5CreateClient?5fail@ 00000001800059e8     sawindbg.obj
 0002:00000a10       ??_C@_0DE@HJKLOPIF@Windbg?5Error?3?5QueryInterface?5?$CII@ 0000000180005a10     sawindbg.obj
 0002:00000a48       ??_C@_0CJ@LPJOGDLF@Windbg?5Error?3?5SetOutputCallback@ 0000000180005a48     sawindbg.obj
 0002:00000a71       ??_C@_00CNPNBAHC@@         0000000180005a71     sawindbg.obj
 0002:00000a74       ??_C@_02MOLJINC@?3?3@      0000000180005a74     sawindbg.obj
 0002:00000a80       ??_7type_info@@6B@         0000000180005a80     MSVCRT:std_type_info_static.obj
 0002:00000a88       _pDefaultRawDllMain        0000000180005a88     MSVCRT:dll_dllmain.obj
 0002:00000a88       _pRawDllMain               0000000180005a88     MSVCRT:dll_dllmain.obj
 0002:00000aa8       ??_7exception@std@@6B@     0000000180005aa8     MSVCRT:throw_bad_alloc.obj
 0002:00000ab8       ??_C@_0BC@EOODALEL@Unknown?5exception@ 0000000180005ab8     MSVCRT:throw_bad_alloc.obj
 0002:00000ad8       ??_7bad_alloc@std@@6B@     0000000180005ad8     MSVCRT:throw_bad_alloc.obj
 0002:00000ae8       ??_C@_0P@GHFPNOJB@bad?5allocation@ 0000000180005ae8     MSVCRT:throw_bad_alloc.obj
 0002:00000b00       ??_7bad_array_new_length@std@@6B@ 0000000180005b00     MSVCRT:throw_bad_alloc.obj
 0002:00000b10       ??_C@_0BF@KINCDENJ@bad?5array?5new?5length@ 0000000180005b10     MSVCRT:throw_bad_alloc.obj
 0002:00000b30       __xmm@ffffffffffffffffffffffffffffffff 0000000180005b30     MSVCRT:utility.obj
 0002:00000b40       _load_config_used          0000000180005b40     MSVCRT:loadcfg.obj
 0002:00000d00       ??_R3IUnknown@@8           0000000180005d00     sawindbg.obj
 0002:00000d18       ??_R2IUnknown@@8           0000000180005d18     sawindbg.obj
 0002:00000d28       ??_R1A@?0A@EA@IUnknown@@8  0000000180005d28     sawindbg.obj
 0002:00000d50       ??_R3IDebugOutputCallbacks@@8 0000000180005d50     sawindbg.obj
 0002:00000d68       ??_R2IDebugOutputCallbacks@@8 0000000180005d68     sawindbg.obj
 0002:00000d80       ??_R1A@?0A@EA@IDebugOutputCallbacks@@8 0000000180005d80     sawindbg.obj
 0002:00000da8       ??_R4SAOutputCallbacks@@6B@ 0000000180005da8     sawindbg.obj
 0002:00000dd0       ??_R3SAOutputCallbacks@@8  0000000180005dd0     sawindbg.obj
 0002:00000de8       ??_R2SAOutputCallbacks@@8  0000000180005de8     sawindbg.obj
 0002:00000e08       ??_R1A@?0A@EA@SAOutputCallbacks@@8 0000000180005e08     sawindbg.obj
 0002:00000e30       ??_R4type_info@@6B@        0000000180005e30     MSVCRT:std_type_info_static.obj
 0002:00000e58       ??_R3type_info@@8          0000000180005e58     MSVCRT:std_type_info_static.obj
 0002:00000e70       ??_R2type_info@@8          0000000180005e70     MSVCRT:std_type_info_static.obj
 0002:00000e80       ??_R1A@?0A@EA@type_info@@8 0000000180005e80     MSVCRT:std_type_info_static.obj
 0002:00000ea8       ??_R4exception@std@@6B@    0000000180005ea8     MSVCRT:throw_bad_alloc.obj
 0002:00000ed0       ??_R3exception@std@@8      0000000180005ed0     MSVCRT:throw_bad_alloc.obj
 0002:00000ee8       ??_R2exception@std@@8      0000000180005ee8     MSVCRT:throw_bad_alloc.obj
 0002:00000ef8       ??_R1A@?0A@EA@exception@std@@8 0000000180005ef8     MSVCRT:throw_bad_alloc.obj
 0002:00000f20       ??_R4bad_alloc@std@@6B@    0000000180005f20     MSVCRT:throw_bad_alloc.obj
 0002:00000f48       ??_R3bad_alloc@std@@8      0000000180005f48     MSVCRT:throw_bad_alloc.obj
 0002:00000f60       ??_R2bad_alloc@std@@8      0000000180005f60     MSVCRT:throw_bad_alloc.obj
 0002:00000f78       ??_R1A@?0A@EA@bad_alloc@std@@8 0000000180005f78     MSVCRT:throw_bad_alloc.obj
 0002:00000fa0       ??_R4bad_array_new_length@std@@6B@ 0000000180005fa0     MSVCRT:throw_bad_alloc.obj
 0002:00000fc8       ??_R3bad_array_new_length@std@@8 0000000180005fc8     MSVCRT:throw_bad_alloc.obj
 0002:00000fe0       ??_R2bad_array_new_length@std@@8 0000000180005fe0     MSVCRT:throw_bad_alloc.obj
 0002:00001000       ??_R1A@?0A@EA@bad_array_new_length@std@@8 0000000180006000     MSVCRT:throw_bad_alloc.obj
 0002:00001024       __volatile_metadata        0000000180006024     <linker-defined>
 0002:00001398       __rtc_iaa                  0000000180006398     MSVCRT:initsect.obj
 0002:000013a0       __rtc_izz                  00000001800063a0     MSVCRT:initsect.obj
 0002:000013a8       __rtc_taa                  00000001800063a8     MSVCRT:initsect.obj
 0002:000013b0       __rtc_tzz                  00000001800063b0     MSVCRT:initsect.obj
 0002:000018e8       _TI2?AVbad_alloc@std@@     00000001800068e8     MSVCRT:throw_bad_alloc.obj
 0002:00001908       _CTA2?AVbad_alloc@std@@    0000000180006908     MSVCRT:throw_bad_alloc.obj
 0002:00001920       _CT??_R0?AVbad_alloc@std@@@8??0bad_alloc@std@@QEAA@AEBV01@@Z24 0000000180006920     MSVCRT:throw_bad_alloc.obj
 0002:00001948       _CT??_R0?AVexception@std@@@8??0exception@std@@QEAA@AEBV01@@Z24 0000000180006948     MSVCRT:throw_bad_alloc.obj
 0002:00001970       _TI3?AVbad_array_new_length@std@@ 0000000180006970     MSVCRT:throw_bad_alloc.obj
 0002:00001990       _CTA3?AVbad_array_new_length@std@@ 0000000180006990     MSVCRT:throw_bad_alloc.obj
 0002:000019b0       _CT??_R0?AVbad_array_new_length@std@@@8??0bad_array_new_length@std@@QEAA@AEBV01@@Z24 00000001800069b0     MSVCRT:throw_bad_alloc.obj
 0002:00001d90       __IMPORT_DESCRIPTOR_dbgeng 0000000180006d90     dbgeng:dbgeng.dll
 0002:00001da4       __IMPORT_DESCRIPTOR_java   0000000180006da4     java:java.dll
 0002:00001db8       __IMPORT_DESCRIPTOR_KERNEL32 0000000180006db8     kernel32:KERNEL32.dll
 0002:00001dcc       __IMPORT_DESCRIPTOR_VCRUNTIME140 0000000180006dcc     vcruntime:VCRUNTIME140.dll
 0002:00001de0       __IMPORT_DESCRIPTOR_VCRUNTIME140_1 0000000180006de0     vcruntime:VCRUNTIME140_1.dll
 0002:00001df4       __IMPORT_DESCRIPTOR_api-ms-win-crt-stdio-l1-1-0 0000000180006df4     ucrt:api-ms-win-crt-stdio-l1-1-0.dll
 0002:00001e08       __IMPORT_DESCRIPTOR_api-ms-win-crt-string-l1-1-0 0000000180006e08     ucrt:api-ms-win-crt-string-l1-1-0.dll
 0002:00001e1c       __IMPORT_DESCRIPTOR_api-ms-win-crt-heap-l1-1-0 0000000180006e1c     ucrt:api-ms-win-crt-heap-l1-1-0.dll
 0002:00001e30       __IMPORT_DESCRIPTOR_api-ms-win-crt-runtime-l1-1-0 0000000180006e30     ucrt:api-ms-win-crt-runtime-l1-1-0.dll
 0002:00001e44       __NULL_IMPORT_DESCRIPTOR   0000000180006e44     dbgeng:dbgeng.dll
 0003:00000000       __security_cookie_complement 0000000180008000     MSVCRT:gs_cookie.obj
 0003:00000008       __security_cookie          0000000180008008     MSVCRT:gs_cookie.obj
 0003:00000010       __scrt_native_dllmain_reason 0000000180008010     MSVCRT:utility.obj
 0003:00000018       __isa_available            0000000180008018     MSVCRT:cpu_disp.obj
 0003:0000001c       __isa_enabled              000000018000801c     MSVCRT:cpu_disp.obj
 0003:00000020       __memset_fast_string_threshold 0000000180008020     MSVCRT:cpu_disp.obj
 0003:00000028       __memset_nt_threshold      0000000180008028     MSVCRT:cpu_disp.obj
 0003:00000030       __scrt_ucrt_dll_is_in_use  0000000180008030     MSVCRT:ucrt_stubs.obj
 0003:00000038       ??_R0?AVbad_alloc@std@@@8  0000000180008038     MSVCRT:throw_bad_alloc.obj
 0003:00000060       ??_R0?AVexception@std@@@8  0000000180008060     MSVCRT:throw_bad_alloc.obj
 0003:00000088       ??_R0?AVbad_array_new_length@std@@@8 0000000180008088     MSVCRT:throw_bad_alloc.obj
 0003:000000b8       ??_R0?AUIUnknown@@@8       00000001800080b8     sawindbg.obj
 0003:000000d8       ??_R0?AUIDebugOutputCallbacks@@@8 00000001800080d8     sawindbg.obj
 0003:00000108       ??_R0?AVSAOutputCallbacks@@@8 0000000180008108     sawindbg.obj
 0003:00000130       ??_R0?AVtype_info@@@8      0000000180008130     MSVCRT:std_type_info_static.obj
 0003:00000730       ?__type_info_root_node@@3U__type_info_node@@A 0000000180008730     MSVCRT:tncleanup.obj
 0003:00000740       ?_OptionsStorage@?1??__local_stdio_scanf_options@@9@4_KA 0000000180008740     MSVCRT:default_local_stdio_options.obj
 0003:00000748       __scrt_current_native_startup_state 0000000180008748     MSVCRT:utility.obj
 0003:00000750       __scrt_native_startup_lock 0000000180008750     MSVCRT:utility.obj
 0003:00000790       __scrt_debugger_hook_flag  0000000180008790     MSVCRT:utility_desktop.obj
 0003:00000794       __favor                    0000000180008794     MSVCRT:cpu_disp.obj
 0003:00000798       ?_OptionsStorage@?1??__local_stdio_printf_options@@9@9 0000000180008798     <common>
 0003:000007a0       __dyn_tls_init_callback    00000001800087a0     <common>

 entry point at        0001:00002b18

 Static symbols

 0000:ffff4000       .debug$S                   0000000180000000     saproc.exp
 0000:ffff4000       .debug$S                   0000000180000000     vcruntime:VCRUNTIME140.dll
 0000:ffff4000       .debug$S                   0000000180000000     vcruntime:VCRUNTIME140.dll
 0000:ffff4000       .debug$S                   0000000180000000     vcruntime:VCRUNTIME140.dll
 0000:ffff4000       .debug$S                   0000000180000000     vcruntime:VCRUNTIME140.dll
 0000:ffff4000       .debug$S                   0000000180000000     vcruntime:VCRUNTIME140.dll
 0000:ffff4000       .debug$S                   0000000180000000     vcruntime:VCRUNTIME140.dll
 0000:ffff4000       .debug$S                   0000000180000000     vcruntime:VCRUNTIME140.dll
 0000:ffff4000       .debug$S                   0000000180000000     vcruntime:VCRUNTIME140.dll
 0000:ffff4000       .debug$S                   0000000180000000     vcruntime:VCRUNTIME140.dll
 0000:ffff4000       .debug$S                   0000000180000000     vcruntime:VCRUNTIME140.dll
 0000:ffff4000       .debug$S                   0000000180000000     vcruntime:VCRUNTIME140.dll
 0000:ffff4000       .debug$S                   0000000180000000     vcruntime:VCRUNTIME140.dll
 0000:ffff4000       .debug$S                   0000000180000000     vcruntime:VCRUNTIME140.dll
 0000:ffff4000       .debug$S                   0000000180000000     vcruntime:VCRUNTIME140_1.dll
 0000:ffff4000       .debug$S                   0000000180000000     ucrt:api-ms-win-crt-heap-l1-1-0.dll
 0000:ffff4000       .debug$S                   0000000180000000     ucrt:api-ms-win-crt-heap-l1-1-0.dll
 0000:ffff4000       .debug$S                   0000000180000000     ucrt:api-ms-win-crt-heap-l1-1-0.dll
 0000:ffff4000       .debug$S                   0000000180000000     ucrt:api-ms-win-crt-heap-l1-1-0.dll
 0000:ffff4000       .debug$S                   0000000180000000     ucrt:api-ms-win-crt-runtime-l1-1-0.dll
 0000:ffff4000       .debug$S                   0000000180000000     ucrt:api-ms-win-crt-runtime-l1-1-0.dll
 0000:ffff4000       .debug$S                   0000000180000000     ucrt:api-ms-win-crt-runtime-l1-1-0.dll
 0000:ffff4000       .debug$S                   0000000180000000     ucrt:api-ms-win-crt-runtime-l1-1-0.dll
 0000:ffff4000       .debug$S                   0000000180000000     ucrt:api-ms-win-crt-runtime-l1-1-0.dll
 0000:ffff4000       .debug$S                   0000000180000000     ucrt:api-ms-win-crt-runtime-l1-1-0.dll
 0000:ffff4000       .debug$S                   0000000180000000     ucrt:api-ms-win-crt-runtime-l1-1-0.dll
 0000:ffff4000       .debug$S                   0000000180000000     ucrt:api-ms-win-crt-runtime-l1-1-0.dll
 0000:ffff4000       .debug$S                   0000000180000000     ucrt:api-ms-win-crt-runtime-l1-1-0.dll
 0000:ffff4000       .debug$S                   0000000180000000     ucrt:api-ms-win-crt-runtime-l1-1-0.dll
 0000:ffff4000       .debug$S                   0000000180000000     ucrt:api-ms-win-crt-runtime-l1-1-0.dll
 0000:ffff4000       .debug$S                   0000000180000000     ucrt:api-ms-win-crt-runtime-l1-1-0.dll
 0000:ffff4000       .debug$S                   0000000180000000     ucrt:api-ms-win-crt-stdio-l1-1-0.dll
 0000:ffff4000       .debug$S                   0000000180000000     ucrt:api-ms-win-crt-stdio-l1-1-0.dll
 0000:ffff4000       .debug$S                   0000000180000000     ucrt:api-ms-win-crt-stdio-l1-1-0.dll
 0000:ffff4000       .debug$S                   0000000180000000     ucrt:api-ms-win-crt-string-l1-1-0.dll
 0000:ffff4000       .debug$S                   0000000180000000     ucrt:api-ms-win-crt-string-l1-1-0.dll
 0000:ffff4000       .debug$S                   0000000180000000     ucrt:api-ms-win-crt-string-l1-1-0.dll
 0000:ffff4000       .debug$S                   0000000180000000     dbgeng:dbgeng.dll
 0000:ffff4000       .debug$S                   0000000180000000     kernel32:KERNEL32.dll
 0000:ffff4000       .debug$S                   0000000180000000     kernel32:KERNEL32.dll
 0000:ffff4000       .debug$S                   0000000180000000     kernel32:KERNEL32.dll
 0000:ffff4000       .debug$S                   0000000180000000     kernel32:KERNEL32.dll
 0000:ffff4000       .debug$S                   0000000180000000     kernel32:KERNEL32.dll
 0000:ffff4000       .debug$S                   0000000180000000     kernel32:KERNEL32.dll
 0000:ffff4000       .debug$S                   0000000180000000     kernel32:KERNEL32.dll
 0000:ffff4000       .debug$S                   0000000180000000     kernel32:KERNEL32.dll
 0000:ffff4000       .debug$S                   0000000180000000     kernel32:KERNEL32.dll
 0000:ffff4000       .debug$S                   0000000180000000     kernel32:KERNEL32.dll
 0000:ffff4000       .debug$S                   0000000180000000     kernel32:KERNEL32.dll
 0000:ffff4000       .debug$S                   0000000180000000     kernel32:KERNEL32.dll
 0000:ffff4000       .debug$S                   0000000180000000     kernel32:KERNEL32.dll
 0000:ffff4000       .debug$S                   0000000180000000     kernel32:KERNEL32.dll
 0000:ffff4000       .debug$S                   0000000180000000     kernel32:KERNEL32.dll
 0000:ffff4000       .debug$S                   0000000180000000     kernel32:KERNEL32.dll
 0000:ffff4000       .debug$S                   0000000180000000     kernel32:KERNEL32.dll
 0000:ffff4000       .debug$S                   0000000180000000     kernel32:KERNEL32.dll
 0000:ffff4000       .debug$S                   0000000180000000     kernel32:KERNEL32.dll
 0000:ffff4000       .debug$S                   0000000180000000     kernel32:KERNEL32.dll
 0000:ffff4000       .debug$S                   0000000180000000     java:java.dll
 0001:000002c8       event_to_env               00000001800012c8 f   sadis.obj
 0001:00000360       printf_to_env              0000000180001360 f   sadis.obj
 0001:000004f0       ??1?$AutoArrayPtr@D@?A0x8a3339d6@@QEAA@XZ 00000001800014f0 f   sawindbg.obj
 0001:000004f0       ??1?$AutoArrayPtr@K@?A0x8a3339d6@@QEAA@XZ 00000001800014f0 f   sawindbg.obj
 0001:000004f0       ??1?$AutoArrayPtr@U_DEBUG_MODULE_PARAMETERS@@@?A0x8a3339d6@@QEAA@XZ 00000001800014f0 f   sawindbg.obj
 0001:000004f8       ??1AutoJavaString@?A0x8a3339d6@@QEAA@XZ 00000001800014f8 f   sawindbg.obj
 0001:000006f4       ?WaitForEvent@@YAJPEAUIDebugControl@@@Z 00000001800016f4 f   sawindbg.obj
 0001:00000748       ?addLoadObjects@@YA_NPEAUJNIEnv_@@PEAV_jobject@@@Z 0000000180001748 f   sawindbg.obj
 0001:00000a58       ?addThreads@@YA_NPEAUJNIEnv_@@PEAV_jobject@@@Z 0000000180001a58 f   sawindbg.obj
 0001:00000f98       ?attachToProcess@@YA_NPEAUJNIEnv_@@PEAV_jobject@@J@Z 0000000180001f98 f   sawindbg.obj
 0001:00001114       ?getWindbgInterfaces@@YA_NPEAUJNIEnv_@@PEAV_jobject@@@Z 0000000180002114 f   sawindbg.obj
 0001:00001510       ?openDumpFile@@YA_NPEAUJNIEnv_@@PEAV_jobject@@PEAV_jstring@@@Z 0000000180002510 f   sawindbg.obj
 0001:000016f8       ?releaseWindbgInterfaces@@YA_NPEAUJNIEnv_@@PEAV_jobject@@@Z 00000001800026f8 f   sawindbg.obj
 0001:000018a4       ?setImageAndSymbolPath@@YA_NPEAUJNIEnv_@@PEAV_jobject@@@Z 00000001800028a4 f   sawindbg.obj
 0001:00001a6c       ?throwNewDebuggerException@@YAXPEAUJNIEnv_@@PEBD@Z 0000000180002a6c f   sawindbg.obj
 0001:00002670       $$000000                   0000000180003670     MSVCRT:chkstk.obj
 0001:000026d0       $$000000                   00000001800036d0     MSVCRT:amdsecgs.obj
 0001:000027f8       ?dllmain_crt_dispatch@@YAHQEAUHINSTANCE__@@KQEAX@Z 00000001800037f8 f   MSVCRT:dll_dllmain.obj
 0001:00002848       ?dllmain_crt_process_attach@@YAHQEAUHINSTANCE__@@QEAX@Z 0000000180003848 f   MSVCRT:dll_dllmain.obj
 0001:00002960       ?dllmain_crt_process_detach@@YAH_N@Z 0000000180003960 f   MSVCRT:dll_dllmain.obj
 0001:000029e4       ?dllmain_dispatch@@YAHQEAUHINSTANCE__@@KQEAX@Z 00000001800039e4 f   MSVCRT:dll_dllmain.obj
 0001:00002c60       capture_previous_context   0000000180003c60 f   MSVCRT:gs_report.obj
 0001:00003700       $$000000                   0000000180004700     MSVCRT:guard_dispatch.obj
 0001:00003720       $$000000                   0000000180004720     MSVCRT:guard_xfg_dispatch.obj
 0001:00003736       ?dtor$0@?0??addLoadObjects@@YA_NPEAUJNIEnv_@@PEAV_jobject@@@Z@4HA 0000000180004736 f   sawindbg.obj
 0001:00003736       ?dtor$2@?0??addLoadObjects@@YA_NPEAUJNIEnv_@@PEAV_jobject@@@Z@4HA 0000000180004736 f   sawindbg.obj
 0001:00003736       ?dtor$3@?0??addLoadObjects@@YA_NPEAUJNIEnv_@@PEAV_jobject@@@Z@4HA 0000000180004736 f   sawindbg.obj
 0001:00003742       ?dtor$1@?0??addLoadObjects@@YA_NPEAUJNIEnv_@@PEAV_jobject@@@Z@4HA 0000000180004742 f   sawindbg.obj
 0001:0000374e       ?dtor$0@?0??addThreads@@YA_NPEAUJNIEnv_@@PEAV_jobject@@@Z@4HA 000000018000474e f   sawindbg.obj
 0001:0000374e       ?dtor$3@?0??addThreads@@YA_NPEAUJNIEnv_@@PEAV_jobject@@@Z@4HA 000000018000474e f   sawindbg.obj
 0001:0000374e       ?dtor$4@?0??addThreads@@YA_NPEAUJNIEnv_@@PEAV_jobject@@@Z@4HA 000000018000474e f   sawindbg.obj
 0001:0000374e       ?dtor$5@?0??addThreads@@YA_NPEAUJNIEnv_@@PEAV_jobject@@@Z@4HA 000000018000474e f   sawindbg.obj
 0001:0000375a       ?dtor$0@?0??attachToProcess@@YA_NPEAUJNIEnv_@@PEAV_jobject@@J@Z@4HA 000000018000475a f   sawindbg.obj
 0001:0000375a       ?dtor$1@?0??addThreads@@YA_NPEAUJNIEnv_@@PEAV_jobject@@@Z@4HA 000000018000475a f   sawindbg.obj
 0001:0000375a       ?dtor$1@?0??attachToProcess@@YA_NPEAUJNIEnv_@@PEAV_jobject@@J@Z@4HA 000000018000475a f   sawindbg.obj
 0001:00003766       ?dtor$2@?0??addThreads@@YA_NPEAUJNIEnv_@@PEAV_jobject@@@Z@4HA 0000000180004766 f   sawindbg.obj
 0001:00003772       ?dtor$0@?0??getWindbgInterfaces@@YA_NPEAUJNIEnv_@@PEAV_jobject@@@Z@4HA 0000000180004772 f   sawindbg.obj
 0001:00003772       ?dtor$1@?0??getWindbgInterfaces@@YA_NPEAUJNIEnv_@@PEAV_jobject@@@Z@4HA 0000000180004772 f   sawindbg.obj
 0001:00003772       ?dtor$2@?0??getWindbgInterfaces@@YA_NPEAUJNIEnv_@@PEAV_jobject@@@Z@4HA 0000000180004772 f   sawindbg.obj
 0001:00003772       ?dtor$4@?0??getWindbgInterfaces@@YA_NPEAUJNIEnv_@@PEAV_jobject@@@Z@4HA 0000000180004772 f   sawindbg.obj
 0001:00003772       ?dtor$5@?0??getWindbgInterfaces@@YA_NPEAUJNIEnv_@@PEAV_jobject@@@Z@4HA 0000000180004772 f   sawindbg.obj
 0001:00003772       ?dtor$6@?0??getWindbgInterfaces@@YA_NPEAUJNIEnv_@@PEAV_jobject@@@Z@4HA 0000000180004772 f   sawindbg.obj
 0001:0000377e       ?dtor$0@?0??openDumpFile@@YA_NPEAUJNIEnv_@@PEAV_jobject@@PEAV_jstring@@@Z@4HA 000000018000477e f   sawindbg.obj
 0001:0000378a       ?dtor$1@?0??openDumpFile@@YA_NPEAUJNIEnv_@@PEAV_jobject@@PEAV_jstring@@@Z@4HA 000000018000478a f   sawindbg.obj
 0001:0000378a       ?dtor$2@?0??openDumpFile@@YA_NPEAUJNIEnv_@@PEAV_jobject@@PEAV_jstring@@@Z@4HA 000000018000478a f   sawindbg.obj
 0001:00003796       ?dtor$0@?0??setImageAndSymbolPath@@YA_NPEAUJNIEnv_@@PEAV_jobject@@@Z@4HA 0000000180004796 f   sawindbg.obj
 0001:000037a2       ?dtor$1@?0??setImageAndSymbolPath@@YA_NPEAUJNIEnv_@@PEAV_jobject@@@Z@4HA 00000001800047a2 f   sawindbg.obj
 0001:000037ae       ?fin$0@?0??dllmain_crt_process_attach@@YAHQEAUHINSTANCE__@@QEAX@Z@4HA 00000001800047ae f   MSVCRT:dll_dllmain.obj
 0001:000037c5       ?fin$0@?0??dllmain_crt_process_detach@@YAH_N@Z@4HA 00000001800047c5 f   MSVCRT:dll_dllmain.obj
 0001:000037de       ?fin$1@?0??dllmain_crt_process_detach@@YAH_N@Z@4HA 00000001800047de f   MSVCRT:dll_dllmain.obj
 0001:000037f2       ?filt$0@?0??dllmain_dispatch@@YAHQEAUHINSTANCE__@@KQEAX@Z@4HA 00000001800047f2 f   MSVCRT:dll_dllmain.obj
 0001:00003828       __scrt_is_nonwritable_in_current_image$filt$0 0000000180004828 f   MSVCRT:utility.obj
 0002:00000a90       GS_ExceptionPointers       0000000180005a90     MSVCRT:gs_report.obj
 0002:000013b8       $unwind$Java_sun_jvm_hotspot_asm_Disassembler_load_1library 00000001800063b8     sadis.obj
 0002:000013b8       $unwind$?Output@SAOutputCallbacks@@UEAAJKPEBD@Z 00000001800063b8     sawindbg.obj
 0002:000013b8       $unwind$__scrt_dllmain_exception_filter 00000001800063b8     MSVCRT:utility.obj
 0002:000013cc       $unwind$Java_sun_jvm_hotspot_asm_Disassembler_decode 00000001800063cc     sadis.obj
 0002:000013ec       $unwind$event_to_env       00000001800063ec     sadis.obj
 0002:00001400       $unwind$printf_to_env      0000000180006400     sadis.obj
 0002:00001410       $unwind$fprintf            0000000180006410     sawindbg.obj
 0002:0000141c       $unwind$printf             000000018000641c     sawindbg.obj
 0002:00001428       $unwind$snprintf           0000000180006428     sawindbg.obj
 0002:00001438       $unwind$?CallObjectMethod@JNIEnv_@@QEAAPEAV_jobject@@PEAV2@PEAU_jmethodID@@ZZ 0000000180006438     sawindbg.obj
 0002:00001438       $unwind$?CallVoidMethod@JNIEnv_@@QEAAXPEAV_jobject@@PEAU_jmethodID@@ZZ 0000000180006438     sawindbg.obj
 0002:00001440       $unwind$?QueryInterface@SAOutputCallbacks@@UEAAJAEBU_GUID@@PEAPEAX@Z 0000000180006440     sawindbg.obj
 0002:00001440       $unwind$?releaseWindbgInterfaces@@YA_NPEAUJNIEnv_@@PEAV_jobject@@@Z 0000000180006440     sawindbg.obj
 0002:00001440       $unwind$?throwNewDebuggerException@@YAXPEAUJNIEnv_@@PEBD@Z 0000000180006440     sawindbg.obj
 0002:00001440       $unwind$Java_sun_jvm_hotspot_debugger_windbg_WindbgDebuggerLocal_attach0__I 0000000180006440     sawindbg.obj
 0002:00001440       $unwind$Java_sun_jvm_hotspot_debugger_windbg_WindbgDebuggerLocal_attach0__Ljava_lang_String_2Ljava_lang_String_2 0000000180006440     sawindbg.obj
 0002:00001440       $unwind$Java_sun_jvm_hotspot_debugger_windbg_WindbgDebuggerLocal_detach0 0000000180006440     sawindbg.obj
 0002:00001440       $unwind$Java_sun_jvm_hotspot_debugger_windbg_WindbgDebuggerLocal_initIDs 0000000180006440     sawindbg.obj
 0002:00001440       $unwind$_DllMainCRTStartup 0000000180006440     MSVCRT:dll_dllmain.obj
 0002:00001450       $unwind$Java_sun_jvm_hotspot_debugger_windbg_WindbgDebuggerLocal_readBytesFromProcess0 0000000180006450     sawindbg.obj
 0002:00001470       $cppxdata$Java_sun_jvm_hotspot_debugger_windbg_WindbgDebuggerLocal_readBytesFromProcess0 0000000180006470     sawindbg.obj
 0002:00001479       $stateUnwindMap$Java_sun_jvm_hotspot_debugger_windbg_WindbgDebuggerLocal_readBytesFromProcess0 0000000180006479     sawindbg.obj
 0002:00001482       $ip2state$Java_sun_jvm_hotspot_debugger_windbg_WindbgDebuggerLocal_readBytesFromProcess0 0000000180006482     sawindbg.obj
 0002:0000148c       $unwind$Java_sun_jvm_hotspot_debugger_windbg_WindbgDebuggerLocal_getThreadIdFromSysId0 000000018000648c     sawindbg.obj
 0002:0000149c       $unwind$Java_sun_jvm_hotspot_debugger_windbg_WindbgDebuggerLocal_consoleExecuteCommand0 000000018000649c     sawindbg.obj
 0002:000014bc       $cppxdata$Java_sun_jvm_hotspot_debugger_windbg_WindbgDebuggerLocal_consoleExecuteCommand0 00000001800064bc     sawindbg.obj
 0002:000014c5       $stateUnwindMap$Java_sun_jvm_hotspot_debugger_windbg_WindbgDebuggerLocal_consoleExecuteCommand0 00000001800064c5     sawindbg.obj
 0002:000014dc       $ip2state$Java_sun_jvm_hotspot_debugger_windbg_WindbgDebuggerLocal_consoleExecuteCommand0 00000001800064dc     sawindbg.obj
 0002:000014ec       $unwind$Java_sun_jvm_hotspot_debugger_windbg_WindbgDebuggerLocal_lookupByName0 00000001800064ec     sawindbg.obj
 0002:00001508       $cppxdata$Java_sun_jvm_hotspot_debugger_windbg_WindbgDebuggerLocal_lookupByName0 0000000180006508     sawindbg.obj
 0002:00001511       $stateUnwindMap$Java_sun_jvm_hotspot_debugger_windbg_WindbgDebuggerLocal_lookupByName0 0000000180006511     sawindbg.obj
 0002:00001519       $ip2state$Java_sun_jvm_hotspot_debugger_windbg_WindbgDebuggerLocal_lookupByName0 0000000180006519     sawindbg.obj
 0002:00001524       $unwind$Java_sun_jvm_hotspot_debugger_windbg_WindbgDebuggerLocal_lookupByAddress0 0000000180006524     sawindbg.obj
 0002:00001540       $unwind$??1AutoJavaString@?A0x8a3339d6@@QEAA@XZ 0000000180006540     sawindbg.obj
 0002:00001550       $cppxdata$??1AutoJavaString@?A0x8a3339d6@@QEAA@XZ 0000000180006550     sawindbg.obj
 0002:00001555       $ip2state$??1AutoJavaString@?A0x8a3339d6@@QEAA@XZ 0000000180006555     sawindbg.obj
 0002:00001558       $unwind$?Release@SAOutputCallbacks@@UEAAKXZ 0000000180006558     sawindbg.obj
 0002:00001558       $unwind$?WaitForEvent@@YAJPEAUIDebugControl@@@Z 0000000180006558     sawindbg.obj
 0002:00001558       $unwind$_RTC_Initialize    0000000180006558     MSVCRT:initsect.obj
 0002:00001558       $unwind$_RTC_Terminate     0000000180006558     MSVCRT:initsect.obj
 0002:00001558       $unwind$??_Gbad_alloc@std@@UEAAPEAXI@Z 0000000180006558     MSVCRT:throw_bad_alloc.obj
 0002:00001558       $unwind$??_Gbad_array_new_length@std@@UEAAPEAXI@Z 0000000180006558     MSVCRT:throw_bad_alloc.obj
 0002:00001558       $unwind$??_Gexception@std@@UEAAPEAXI@Z 0000000180006558     MSVCRT:throw_bad_alloc.obj
 0002:00001564       $unwind$?getWindbgInterfaces@@YA_NPEAUJNIEnv_@@PEAV_jobject@@@Z 0000000180006564     sawindbg.obj
 0002:00001580       $cppxdata$?getWindbgInterfaces@@YA_NPEAUJNIEnv_@@PEAV_jobject@@@Z 0000000180006580     sawindbg.obj
 0002:00001589       $stateUnwindMap$?getWindbgInterfaces@@YA_NPEAUJNIEnv_@@PEAV_jobject@@@Z 0000000180006589     sawindbg.obj
 0002:00001590       $ip2state$?getWindbgInterfaces@@YA_NPEAUJNIEnv_@@PEAV_jobject@@@Z 0000000180006590     sawindbg.obj
 0002:000015ac       $unwind$?setImageAndSymbolPath@@YA_NPEAUJNIEnv_@@PEAV_jobject@@@Z 00000001800065ac     sawindbg.obj
 0002:000015d0       $cppxdata$?setImageAndSymbolPath@@YA_NPEAUJNIEnv_@@PEAV_jobject@@@Z 00000001800065d0     sawindbg.obj
 0002:000015d9       $stateUnwindMap$?setImageAndSymbolPath@@YA_NPEAUJNIEnv_@@PEAV_jobject@@@Z 00000001800065d9     sawindbg.obj
 0002:000015f7       $ip2state$?setImageAndSymbolPath@@YA_NPEAUJNIEnv_@@PEAV_jobject@@@Z 00000001800065f7     sawindbg.obj
 0002:0000160c       $unwind$?openDumpFile@@YA_NPEAUJNIEnv_@@PEAV_jobject@@PEAV_jstring@@@Z 000000018000660c     sawindbg.obj
 0002:0000162c       $cppxdata$?openDumpFile@@YA_NPEAUJNIEnv_@@PEAV_jobject@@PEAV_jstring@@@Z 000000018000662c     sawindbg.obj
 0002:00001635       $stateUnwindMap$?openDumpFile@@YA_NPEAUJNIEnv_@@PEAV_jobject@@PEAV_jstring@@@Z 0000000180006635     sawindbg.obj
 0002:0000164f       $ip2state$?openDumpFile@@YA_NPEAUJNIEnv_@@PEAV_jobject@@PEAV_jstring@@@Z 000000018000664f     sawindbg.obj
 0002:00001664       $unwind$?attachToProcess@@YA_NPEAUJNIEnv_@@PEAV_jobject@@J@Z 0000000180006664     sawindbg.obj
 0002:00001680       $cppxdata$?attachToProcess@@YA_NPEAUJNIEnv_@@PEAV_jobject@@J@Z 0000000180006680     sawindbg.obj
 0002:00001689       $stateUnwindMap$?attachToProcess@@YA_NPEAUJNIEnv_@@PEAV_jobject@@J@Z 0000000180006689     sawindbg.obj
 0002:00001690       $ip2state$?attachToProcess@@YA_NPEAUJNIEnv_@@PEAV_jobject@@J@Z 0000000180006690     sawindbg.obj
 0002:0000169c       $unwind$?addLoadObjects@@YA_NPEAUJNIEnv_@@PEAV_jobject@@@Z 000000018000669c     sawindbg.obj
 0002:000016c4       $cppxdata$?addLoadObjects@@YA_NPEAUJNIEnv_@@PEAV_jobject@@@Z 00000001800066c4     sawindbg.obj
 0002:000016cd       $stateUnwindMap$?addLoadObjects@@YA_NPEAUJNIEnv_@@PEAV_jobject@@@Z 00000001800066cd     sawindbg.obj
 0002:000016e0       $ip2state$?addLoadObjects@@YA_NPEAUJNIEnv_@@PEAV_jobject@@@Z 00000001800066e0     sawindbg.obj
 0002:000016f8       $unwind$?addThreads@@YA_NPEAUJNIEnv_@@PEAV_jobject@@@Z 00000001800066f8     sawindbg.obj
 0002:00001720       $cppxdata$?addThreads@@YA_NPEAUJNIEnv_@@PEAV_jobject@@@Z 0000000180006720     sawindbg.obj
 0002:00001729       $stateUnwindMap$?addThreads@@YA_NPEAUJNIEnv_@@PEAV_jobject@@@Z 0000000180006729     sawindbg.obj
 0002:00001742       $ip2state$?addThreads@@YA_NPEAUJNIEnv_@@PEAV_jobject@@@Z 0000000180006742     sawindbg.obj
 0002:00001760       $unwind$__GSHandlerCheckCommon 0000000180006760     MSVCRT:gshandler.obj
 0002:00001768       $unwind$__scrt_initialize_default_local_stdio_options 0000000180006768     MSVCRT:default_local_stdio_options.obj
 0002:00001768       $unwind$?dllmain_crt_dispatch@@YAHQEAUHINSTANCE__@@KQEAX@Z 0000000180006768     MSVCRT:dll_dllmain.obj
 0002:00001768       $unwind$DllMain            0000000180006768     MSVCRT:dll_dllmain_stub.obj
 0002:00001768       $unwind$__GSHandlerCheck   0000000180006768     MSVCRT:gshandler.obj
 0002:00001768       $unwind$__scrt_acquire_startup_lock 0000000180006768     MSVCRT:utility.obj
 0002:00001768       $unwind$__scrt_dllmain_after_initialize_c 0000000180006768     MSVCRT:utility.obj
 0002:00001768       $unwind$__scrt_dllmain_before_initialize_c 0000000180006768     MSVCRT:utility.obj
 0002:00001768       $unwind$__scrt_dllmain_crt_thread_attach 0000000180006768     MSVCRT:utility.obj
 0002:00001768       $unwind$__scrt_dllmain_crt_thread_detach 0000000180006768     MSVCRT:utility.obj
 0002:00001768       $unwind$__scrt_dllmain_uninitialize_c 0000000180006768     MSVCRT:utility.obj
 0002:00001768       $unwind$__scrt_dllmain_uninitialize_critical 0000000180006768     MSVCRT:utility.obj
 0002:00001770       $xdatasym                  0000000180006770     MSVCRT:chkstk.obj
 0002:00001778       $xdatasym                  0000000180006778     MSVCRT:amdsecgs.obj
 0002:0000177c       $unwind$__raise_securityfailure 000000018000677c     MSVCRT:gs_report.obj
 0002:0000177c       $unwind$??2@YAPEAX_K@Z     000000018000677c     MSVCRT:new_scalar.obj
 0002:0000177c       $unwind$??_Gtype_info@@UEAAPEAXI@Z 000000018000677c     MSVCRT:std_type_info_static.obj
 0002:0000177c       $unwind$??0bad_alloc@std@@QEAA@AEBV01@@Z 000000018000677c     MSVCRT:throw_bad_alloc.obj
 0002:0000177c       $unwind$??0bad_array_new_length@std@@QEAA@AEBV01@@Z 000000018000677c     MSVCRT:throw_bad_alloc.obj
 0002:0000177c       $unwind$??0exception@std@@QEAA@AEBV01@@Z 000000018000677c     MSVCRT:throw_bad_alloc.obj
 0002:0000177c       $unwind$__scrt_initialize_crt 000000018000677c     MSVCRT:utility.obj
 0002:0000177c       $unwind$__scrt_initialize_onexit_tables 000000018000677c     MSVCRT:utility.obj
 0002:0000177c       $unwind$__scrt_release_startup_lock 000000018000677c     MSVCRT:utility.obj
 0002:0000177c       $unwind$__scrt_uninitialize_crt 000000018000677c     MSVCRT:utility.obj
 0002:00001784       $unwind$__GSHandlerCheck_EH4 0000000180006784     MSVCRT:gshandlereh4.obj
 0002:0000179c       $unwind$?dllmain_crt_process_attach@@YAHQEAUHINSTANCE__@@QEAX@Z 000000018000679c     MSVCRT:dll_dllmain.obj
 0002:000017d8       $unwind$?fin$0@?0??dllmain_crt_process_attach@@YAHQEAUHINSTANCE__@@QEAX@Z@4HA 00000001800067d8     MSVCRT:dll_dllmain.obj
 0002:000017d8       $unwind$?fin$0@?0??dllmain_crt_process_detach@@YAH_N@Z@4HA 00000001800067d8     MSVCRT:dll_dllmain.obj
 0002:000017d8       $unwind$?fin$1@?0??dllmain_crt_process_detach@@YAH_N@Z@4HA 00000001800067d8     MSVCRT:dll_dllmain.obj
 0002:000017e0       $unwind$?dllmain_crt_process_detach@@YAH_N@Z 00000001800067e0     MSVCRT:dll_dllmain.obj
 0002:00001834       $unwind$?dllmain_dispatch@@YAHQEAUHINSTANCE__@@KQEAX@Z 0000000180006834     MSVCRT:dll_dllmain.obj
 0002:0000185c       $unwind$?filt$0@?0??dllmain_dispatch@@YAHQEAUHINSTANCE__@@KQEAX@Z@4HA 000000018000685c     MSVCRT:dll_dllmain.obj
 0002:00001864       $unwind$__report_gsfailure 0000000180006864     MSVCRT:gs_report.obj
 0002:0000186c       $unwind$capture_previous_context 000000018000686c     MSVCRT:gs_report.obj
 0002:00001878       $unwind$?__scrt_throw_std_bad_alloc@@YAXXZ 0000000180006878     MSVCRT:throw_bad_alloc.obj
 0002:00001878       $unwind$?__scrt_throw_std_bad_array_new_length@@YAXXZ 0000000180006878     MSVCRT:throw_bad_alloc.obj
 0002:00001880       $unwind$__security_init_cookie 0000000180006880     MSVCRT:gs_support.obj
 0002:0000188c       $unwind$__scrt_is_nonwritable_in_current_image 000000018000688c     MSVCRT:utility.obj
 0002:000018ac       $unwind$__scrt_is_nonwritable_in_current_image$filt$0 00000001800068ac     MSVCRT:utility.obj
 0002:000018b4       $unwind$__scrt_fastfail    00000001800068b4     MSVCRT:utility_desktop.obj
 0002:000018c4       $unwind$__isa_available_init 00000001800068c4     MSVCRT:cpu_disp.obj
 0002:000018d8       $xdatasym                  00000001800068d8     MSVCRT:guard_dispatch.obj
 0002:000018e0       $xdatasym                  00000001800068e0     MSVCRT:guard_xfg_dispatch.obj
 0002:000019e0       .edata                     00000001800069e0     saproc.exp
 0002:00001a08       rgpv                       0000000180006a08     saproc.exp
 0002:00001a34       rgszName                   0000000180006a34     saproc.exp
 0002:00001a60       rgwOrd                     0000000180006a60     saproc.exp
 0002:00001a76       szName                     0000000180006a76     saproc.exp
 0002:00001a81       $N00001                    0000000180006a81     saproc.exp
 0002:00001aae       $N00002                    0000000180006aae     saproc.exp
 0002:00001ae2       $N00003                    0000000180006ae2     saproc.exp
 0002:00001b26       $N00004                    0000000180006b26     saproc.exp
 0002:00001b8f       $N00005                    0000000180006b8f     saproc.exp
 0002:00001bdf       $N00006                    0000000180006bdf     saproc.exp
 0002:00001c20       $N00007                    0000000180006c20     saproc.exp
 0002:00001c6f       $N00008                    0000000180006c6f     saproc.exp
 0002:00001cb0       $N00009                    0000000180006cb0     saproc.exp
 0002:00001cfa       $N00010                    0000000180006cfa     saproc.exp
 0002:00001d41       $N00011                    0000000180006d41     saproc.exp
 0002:0000203e       .idata$6                   000000018000703e     dbgeng:dbgeng.dll
 0002:0000206a       .idata$6                   000000018000706a     java:java.dll
 0002:0000220e       .idata$6                   000000018000720e     kernel32:KERNEL32.dll
 0002:000022ec       .idata$6                   00000001800072ec     vcruntime:VCRUNTIME140.dll
 0002:000022fe       .idata$6                   00000001800072fe     vcruntime:VCRUNTIME140_1.dll
 0002:00002444       .idata$6                   0000000180007444     ucrt:api-ms-win-crt-stdio-l1-1-0.dll
 0002:00002464       .idata$6                   0000000180007464     ucrt:api-ms-win-crt-string-l1-1-0.dll
 0002:00002486       .idata$6                   0000000180007486     ucrt:api-ms-win-crt-heap-l1-1-0.dll
 0002:000024a6       .idata$6                   00000001800074a6     ucrt:api-ms-win-crt-runtime-l1-1-0.dll
 0003:00000150       ?imagePath_ID@@3PEAU_jfieldID@@EA 0000000180008150     sawindbg.obj
 0003:00000158       ?symbolPath_ID@@3PEAU_jfieldID@@EA 0000000180008158     sawindbg.obj
 0003:00000160       ?ptrIDebugClient_ID@@3PEAU_jfieldID@@EA 0000000180008160     sawindbg.obj
 0003:00000168       ?ptrIDebugControl_ID@@3PEAU_jfieldID@@EA 0000000180008168     sawindbg.obj
 0003:00000170       ?ptrIDebugDataSpaces_ID@@3PEAU_jfieldID@@EA 0000000180008170     sawindbg.obj
 0003:00000178       ?ptrIDebugOutputCallbacks_ID@@3PEAU_jfieldID@@EA 0000000180008178     sawindbg.obj
 0003:00000180       ?ptrIDebugAdvanced_ID@@3PEAU_jfieldID@@EA 0000000180008180     sawindbg.obj
 0003:00000188       ?ptrIDebugSymbols_ID@@3PEAU_jfieldID@@EA 0000000180008188     sawindbg.obj
 0003:00000190       ?ptrIDebugSystemObjects_ID@@3PEAU_jfieldID@@EA 0000000180008190     sawindbg.obj
 0003:00000198       ?addLoadObject_ID@@3PEAU_jmethodID@@EA 0000000180008198     sawindbg.obj
 0003:000001a0       ?addThread_ID@@3PEAU_jmethodID@@EA 00000001800081a0     sawindbg.obj
 0003:000001a8       ?createClosestSymbol_ID@@3PEAU_jmethodID@@EA 00000001800081a8     sawindbg.obj
 0003:000001b0       ?setThreadIntegerRegisterSet_ID@@3PEAU_jmethodID@@EA 00000001800081b0     sawindbg.obj
 0003:000001b8       ?__proc_attached@@3HA      00000001800081b8     MSVCRT:dll_dllmain.obj
 0003:000001c0       GS_ExceptionRecord         00000001800081c0     MSVCRT:gs_report.obj
 0003:00000260       GS_ContextRecord           0000000180008260     MSVCRT:gs_report.obj
 0003:00000758       ?is_initialized_as_dll@@3_NA 0000000180008758     MSVCRT:utility.obj
 0003:00000759       ?module_local_atexit_table_initialized@@3_NA 0000000180008759     MSVCRT:utility.obj
 0003:00000760       ?module_local_atexit_table@@3U_onexit_table_t@@A 0000000180008760     MSVCRT:utility.obj
 0003:00000778       ?module_local_at_quick_exit_table@@3U_onexit_table_t@@A 0000000180008778     MSVCRT:utility.obj
 0005:00000060       $R000000                   000000018000a060     saproc.dll.res
